:020000040000FA
:040000004BEF01F0D1
:10000800D8CF00F0E0CF01F0026EE9CF03F0EACFDD
:1000180004F0FACF05F0FBCF06F0F2A818D0F2A250
:1000280016D0F292F29879A68B94E80ECF6E900EC5
:10003800CE6E9E90CD809D987888789A78A407D0C7
:1000480079BA05D00D0E756002D0020E75269DA8EE
:1000580027D09EA825D09D98788881A021D0799016
:1000680079BA09D0B06A2F0E7C6E81B002D079803F
:1000780002D07C2EFAD779B013D06750E96E020E01
:100088006824EA6EEFCFADFF798A672A000E6822EE
:10009800676605D0020E686202D0676A686A7006F1
:1000A8009DAA72D09EAA70D0F2927888E80ECF6E80
:1000B800900ECE6E9E90CD80ABA203D0AB98AB884D
:1000C80063D0ABA41CD0AE50E20ECF6EB40ECE6E91
:1000D8009E90CD8078AC04D04A0EAF6E789C54D0F8
:1000E80079AA52D0799A788E7C0EAF6EAD6A788CE8
:1000F800D60ECF6EFC0ECE6E9E90CD8045D001EE12
:1001080080F06650E926AECFEFFF78AC04D04A0EF7
:10011800AF6E789C2FD079AA2DD06D50E96E020E63
:100128006E24EA6EEFCF7AF001EE80F06650E92691
:10013800EF507A6213D06D2A000E6E226D6605D0DC
:10014800020E6E6202D06D6A6E6A706605D0799A88
:100158007894756AF2880ED09D880CD0799A788E3A
:100168007C0EAF6EAD6A788CD60ECF6EFC0ECE6E5E
:100178009E90CD805F0E726007D078BC05D0662A4D
:10018800600E666201D0666A9EA053D09E9078A8E1
:100198004CD07898F28879A68B8475C07BF07B4622
:1001A8007B467B44060FF924D8B0FA2AF96EE80E8C
:1001B800CF6E900E36D0E90ECF6EBC0E32D0EA0E5E
:1001C800CF6EE80E2ED0EC0ECF6E140E2AD0ED0EA8
:1001D800CF6E400E26D0EE0ECF6E6C0E22D0EF0EF4
:1001E800CF6E980E1ED0F00ECF6EC40E1AD0F10E40
:1001F800CF6EF00E16D0F30ECF6E1C0E12D0F40E8A
:10020800CF6E480E0ED0F50ECF6E740E0AD0F60ED5
:10021800CF6EA00E06D0F70ECF6ECC0E02D0F80E21
:10022800CF6ECE6ECD80788A04D078AA02D0789A24
:10023800CD909EA21ED09E922682572A130E5764F6
:1002480018D0576A2684582A010E586402D0586A72
:100258002686592A130E59640CD0596A26885A2AB8
:10026800090E5A6406D05A6A268A5B2A0A0E5B600F
:100278005B6A05C0FAFF06C0FBFF03C0E9FF04C0C4
:10028800EAFF025001C0E0FF00C0D8FF100052ECA6
:1002980011F085EC11F0CCEC11F00001FFEC11F03D
:1002A8000400D180F28CF28ECA8478B634D06550BE
:1002B800665C076E07AE02D0600E072607C072F0B4
:1002C800075259E001EE80F06550E926EFAE1ED0E6
:1002D800800E096E010E0A6E65C00BF00C6A0BBE2B
:1002E8000C0607C00DF00E6A0DBE0E06600E0F6EEE
:1002F800106AF0EC09F0716E71503DE0FF0A03E1FD
:10030800B7EC0EF038D0F288788635D0B7EC0EF01E
:10031800072ED8D730D001EE80F06550E926EF508F
:10032800830A0BE0330A0CE0010A14E0030A16E022
:10033800060A18E05B0A19E01BD083EC0EF01AD00D
:10034800000E65EC0CF00FC008F010C009F023ECAB
:100358000BF010D0010E65EC0CF00CD0020E65EC21
:100368000CF008D00AEC10F005D006EC0FF002D023
:10037800B7EC0EF0789626A249D1269278B44DD0E3
:1003880078B84BD06750695C076E68506A58086E39
:1003980008AE02D0020E0826075008103EE067504B
:1003A800E96E020E6824EA6EEFAE2FD0096A020EDB
:1003B8000A6E67C00BF068C00CF007C00DF008C0EB
:1003C8000EF00F6A106EF0EC09F0706E705025E0B8
:1003D800FF0A03E1C2EC0EF020D06750E96E020E6E
:1003E8006824EA6EB20EEF6203D0060E756E01D075
:1003F800756A67C06BF068C06CF070C06FF067C05A
:100408006DF068C06EF0788408D0C2EC0EF0070674
:10041800000E085A07500810C2E178A413D078AE2D
:100428000BD0789E6BC067F06CC068F06FC070F03E
:1004380067C06DF068C06EF079A804D078B802D0B3
:1004480078AA9D8810EEB0F0096A080E0960DED01F
:10045800E6500F90E7BC0F800F92E7BA0F82E6BE16
:10046800D3D0EA6A470E0924E96EEF50D8B4CCD04D
:1004780024EE00F0200E0902F350D9260E6A010E70
:100488000A6E0A52D8B4B7D0EA6A470E0924E96E50
:100498000A50EF14D8B4A9D0EA6A470E0924E96EC5
:1004A8000A1CEF16DECF0DF0DECF0BF079A22ED0AE
:1004B8000FB22CD00D38030B25E10FA006D00EA0EB
:1004C80004D0020ED9260E2A93D0020EE15EE6CFA2
:1004D80007F0E6CF08F00F94EA6A370E0924E96EB0
:1004E8000A50EF14D8A40F8408960FB40886100E8B
:1004F800136E1990199207C014F008C015F00E5029
:1005080071EC0AF0020ED9260E2A72D00F0E0B14C7
:100518000C6E0B38070B0B6E0B5006E0010A04E05B
:10052800030A02E0010A63E10BC010F00CC011F0ED
:100538000DC012F00EC013F009C014F00A50F5EC0B
:1005480008F006E3EA6A800E0924E96E0A50EF1201
:100558000B5203E0020E0B620ED00C520CE0EA6A5A
:100568002F0E0924E96E0A50EF1405E10FA003D0FD
:10057800020ED9263CD0DE5079A202D0DE5037D008
:10058800DEBE35D0D8900D32D8900D32030E0D1442
:10059800010A05E0030A11E0010A20E028D0EA6A0E
:1005A8002F0E0924E96E0A50EF1421E0EA6AA00E22
:1005B8000924E96E0A50EF121AD0EA6A2F0E0924AC
:1005C800E96E0A50EF1413E1E550E6BC10D0EA6A70
:1005D800A00E0924E96E0A50EF1209D0EA6AA00EAB
:1005E8000924E96E0A50EF1202D0040ED9260E2A09
:1005F800D8900A3646D709C024F0EA6A2F0E092493
:10060800E96EEF50C1EC10F0092A1FD726A476D066
:100618002694040078A006D05D2E04D07890000EB1
:10062800C2EC07F081B008D079A80DD0732A140E57
:10063800736209D0799807D0736A79B804D0746660
:1006480002D0010E746E74520FE0742A330E746275
:100658000BD0746AF29EF292F288AB889E9A9D8AB9
:100668009D98AC8AF28E798810EEB0F0076A080E71
:10067800076044D0E650E6AE3FD0EA6A370E07245A
:10068800E96EEFCF09F00750ADEC10F00A6EEA6A98
:100698002F0E0724E96E0AC0EFFFEA6A4F0E0724FF
:1006A800E96EEFCF0CF0EA6A800E0724E96EEFCF0F
:1006B8000DF00A5009180B6E010E086E085216E06C
:1006C80008500D1410E10C500B1408140CE0EA6AE1
:1006D800370E0724E96E0850EF1AEA6A470E072416
:1006E800E96E0850EF12D8900836E8D7EA6A4F0E3C
:1006F8000724E96E0BC0EFFF072AB9D726A6A8D3AF
:1007080026960A6A080E0A6056D1EA6A980E0A24E2
:10071800E96EEF50D8B44DD124EE00F0200E0A0255
:10072800F350D9260D90076A010E0B6E0B52D8B400
:1007380035D1EA6A980E0A24E96E0B50EF14D8B442
:1007480027D1DECF09F0DDCF0CF00C38070B086E8F
:1007580001EE00F0080E0A02F3500724D890E8349E
:10076800E926EE06000EEF5A01EE00F0080E0A0226
:10077800F3500724D890E834E926EE50EF10D8A4B7
:1007880007D1E26AD8900A34B10FE16EE7BED4D03F
:10079800E7AA17D0050ED9260C38F00B0C6E0F0EF1
:1007A800DF140C26050ED95E08C00EF00CC00FF041
:1007B80007C010F00AC011F00B5065EC08F00D806E
:1007C800E7D0EA6AA80E0A24E96E0B50EF1433E06A
:1007D800EA6A980E0A24E96E0B1CEF16EA6A800E84
:1007E8000A24E96E0B50EF1413E008C010F00F0E46
:1007F8000C14116E126A07C013F00AC014F00B50E3
:10080800F5EC08F0EA6A800E0A24E96E0B1CEF1674
:10081800EA6AA80E0A24E96E0B1CEF16EA6A270E8C
:100828000A24E96E0B50EF12EA6AA00E0A24E96E58
:100838000B50EF12ADD00850020A03E0030E086215
:100848001CD0EA6A980E0A24E96E0B1CEF1608C041
:1008580010F00F0E0C14116E126A07C013F00AC0C4
:1008680014F00B50F5EC08F006E3EA6A800E0A244F
:10087800E96E0B50EF120D8028D0085202E0082CC8
:1008880024D0EA6A980E0A24E96E0B1CEF16EA6A6D
:10089800800E0A24E96E0B1CEF16DFBC08D0EA6A4A
:1008A8002F0E0A24E96E0B1CEF160D800ED0EA6A93
:1008B800370E0A24E96E0B50EF1407E1EA6A2F0E8F
:1008C8000A24E96E0B1CEF160D8079B261D0030E75
:1008D800D926DFBE2ED0D8900932D8900932091413
:1008E800010A05E0030A11E0010A1DE022D0EA6AC4
:1008F8002F0E0A24E96E0B50EF141BE0EA6AA00ED3
:100908000A24E96E0B50EF1214D0EA6A2F0E0A245B
:10091800E96E0B50EF140DE1EA6AA00E0A24E96EA5
:100928000B50EF1206D0EA6AA00E0A24E96E0B50AB
:10093800EF12030ED95E2CD0EA6A980E0A24E96EEB
:100948000B1CEF16EA6A270E0A24E96E0B50EF1209
:10095800EA6AA80E0A24E96E0B50EF1413E0EA6A5B
:10096800A80E0A24E96E0B1CEF16EA6AA00E0A24E8
:10097800E96E0B50EF12EA6A800E0A24E96E0B1C2E
:10098800EF1606D0EA6A470E0A24E96E0B50EF12FA
:10099800040ED926072AD8900B36C8D60DA009D040
:1009A8000AC024F0EA6A2F0E0A24E96EEF50C1EC5F
:1009B80010F00A2AA7D610EEB0F00D6A080E0D60E6
:1009C80080D1D8900D340F6EE6CF07F0E6CF08F04F
:1009D80008AE75D16750695C096E68506A580A6E2E
:1009E8000AAE02D0020E0A26EA6A470E0D24E96E04
:1009F800EF50D8B464D10ABE06D0C00E095C010E0F
:100A08000A58D8B05CD124EE00F0200E0D02F35045
:100A1800D926040ED95E000EDA5A1068010E0E6E41
:100A28000E52D8B44CD1040ED926000EDA22102A60
:100A3800EA6A470E0D24E96E0E50EF14D8B43CD183
:100A4800EA6A470E0D24E96E0E1CEF16DECF0BF096
:100A5800DDCF0CF01290EA6A370E0D24E96E0E50C5
:100A6800EF14D8A41280089612B008860B38030B2E
:100A780037E179B221D1089812B00888EA6A270EBE
:100A88000D24E96E0E50EF14D8B48BD0EA6A270E05
:100A98000D24E96E0E1CEF160896EA6A3F0E0D2427
:100AA800E96E0E50EF140888D8B408980BC013F0FC
:100AB8001990199207C014F008C015F0105071EC85
:100AC8000AF0EA6AA00E0D24E96E0E50EF14D8A4BD
:100AD800F3D0EA6A800E0D24E96E0E1CEF16ECD0F6
:100AE8000C38070B5EE179B25CD0EA6A270E0D2458
:100AF800E96E0E50EF1416E0EA6A270E0D24E96E2F
:100B08000E1CEF16EA6A880E0D24E96E0E50EF14DB
:100B1800D880D8B4D89003E212B0CED042D012B068
:100B280040D0CAD0EA6A980E0D24E96E0E50EF1430
:100B380022E1EA6A880E0D24E96E0E1CEF1612A057
:100B480010D00E50EF12030E0B14030A2AE00CC04B
:100B580013F010C014F00DC015F00E50BBEC09F0E6
:100B6800ABD00CC013F010C014F00DC015F00E502F
:100B7800BBEC09F0A1D0EA6A880E0D24E96E0E508C
:100B8800EF14D880D8B4D89003E212B003D009D0BB
:100B980012B007D0EA6A980E0D24E96E0E1CEF1603
:100BA8008BD0030E0B14010A07E0030A08E0010AC0
:100BB80008E0030A54E005D012B003D050D012B0B8
:100BC8004ED00B38030B40E1EA6A980E0D24E96E0B
:100BD8000E50EF1471E1EA6A3F0E0D24E96EEFCF73
:100BE80011F008AC03D00E50111A07D010A003D092
:100BF8000E50111202D00E1C11160E501114088836
:100C0800D8B40898EA6A3F0E0D24E96E11C0EFFFC8
:100C18000C38070B020A09E10CC013F010C014F0DD
:100C28000DC015F00E50A3DB08D0200E136E10C0B7
:100C380014F00DC015F00E509ADB0886EA6A800E93
:100C48000D24E96E0E50EF120BC013F01990199293
:100C580007C014F008C015F0105071EC0AF079B212
:100C68002BD0D8900B32D8900B32030E0B14010AFC
:100C780007E0030A08E0010A08E0030A1DE005D0BE
:100C880012B003D019D012B017D0EA6AA00E0D2402
:100C9800E96E0E50EF12030ED926000EDA22DF3865
:100CA800030B06E1EA6A800E0D24E96E0E50EF127E
:100CB800030ED95E000EDA5AD8900E36B1D60D2A38
:100CC8007DD60E6A080E0E60B3D06750695C096E57
:100CD80068506A580A6E0AAE02D0020E0A26EA6AFC
:100CE800A00E0E24E96EEF50D8B4A0D00ABE06D0EC
:100CF800E00E095C010E0A58D8B098D0E26AD89084
:100D08000E34B10FE16E24EE00F0200E0E02F35007
:100D1800D926116A010E0F6E0F52D8B487D0EA6A2D
:100D2800470E0E24E96E0F50EF147AE1EA6AA00E1E
:100D38000E24E96E0F50EF1473E0E7AE07D0EA6AAD
:100D4800980E0E24E96E0F50EF146DE1EA6AA00EBA
:100D58000E24E96E0F1CEF16DECF0BF0DECF0DF080
:100D6800DECF07F0DECF08F0040ED95E08C00CF025
:100D78000898EA6A370E0E24E96E0F50EF14D8A4CB
:100D880008880C38030B42E1EA6A270E0E24E96E44
:100D98000F50EF1408E0EA6A270E0E24E96E0F1CC4
:100DA800EF16089825D0E7AE14D00B38030B020ACB
:100DB80010E1EA6A3F0E0E24E96E0F1CEF16E7AC4D
:100DC80008D008A806D0EA6A3F0E0E24E96E0F5034
:100DD800EF12200E136E11C014F00EC015F00F5054
:100DE800C6DA0888EA6AA80E0E24E96E0F50EF12D8
:100DF800E7AE07D0EA6A3F0E0E24E96E0F50EF14F3
:100E080001D0000E000A088AD8B4089A0CC013F062
:100E18001990198207C014F008C015F011505DDB55
:100E2800040ED926112AD8900F3676D70E2A4AD71B
:100E380079A20ED0076A080E076007D0EA6A470E43
:100E48000724E96EEF10072AF6D7FF0AD8A479928B
:100E580026A862D026985E520DE05E060F0E5E143C
:100E680009E15E3A5E060F0E5E1403E0140E86D8A2
:100E78005E8A5E3A5F5206E05F2E04D0640E7ED82A
:100E88000A0E5F6E79A42CD076060F0E761428E130
:100E9800763A0F0E7614076E080E07601DD0010E05
:100EA800086E075005E0096ED8900836092EFCD761
:100EB8000850601407E0EA6A470E0724E96EEF68F5
:100EC800798208D0C2A906D0EA6A470E0724E96EDB
:100ED800EF687982762A01D07994763A0A0E7612EA
:100EE80082B219D05C2A79B607D00A0E5C620BD0A0
:100EF8007986010E5F6E07D0020E5C6204D0799687
:100F08005F6A650E5C6E640E5C6203D0D19000EF80
:100F180000F0000101D05C6A26AA59EF01F0269A78
:100F280026AC59EF01F05B04076E080E076059EF15
:100F380001F0E26AD8900734B10FE16EE7AE0FD046
:100F480007506124196E000E62201A6EEA6A3F0E7D
:100F58000724E96EEF50F7EC10F059EF01F0075055
:100F68006124196E000E62201A6EEA6A370E072491
:100F7800E96EEF50F7EC10F059EF01F0246E2452AF
:100F880005E024C05DF078808B9001D08B80120042
:100F98001C6E010EEA6E1BC0E9FF1C461C461C4471
:100FA800060FF924D8B0FA2AF96EEF6A000E00008D
:100FB8003BD00A0EEF6E000E37D0140EEF6E000E07
:100FC80033D0230EEF6E000E2FD0320EEF6E000ED0
:100FD8002BD0410EEF6E000E27D0500EEF6E000E94
:100FE80023D0640EEF6E000E1FD07D0EEF6E000E44
:100FF8001BD0960EEF6E000E17D0C80EEF6E000EC7
:1010080013D02C0EEF6E010E0FD0900EEF6E010E66
:101018000BD0F40EEF6E010E07D0580EEF6E020ED5
:1010280003D0200EEF6E030EEC6E12001B6E010E45
:10103800EA6E1AC0E9FF1B461B46F9501B44F92605
:10104800E80EEF6E030E3BD0DC0EEF6E050E37D0C8
:10105800D00EEF6E070E33D0B80EEF6E0B0E2FD0FA
:10106800A00EEF6E0F0E2BD0880EEF6E130E27D04A
:10107800700EEF6E170E23D0280EEF6E230E1FD0C2
:10108800E00EEF6E2E0E1BD0500EEF6E460E17D0F0
:10109800C00EEF6E5D0E13D0300EEF6E750E0FD0D2
:1010A800A00EEF6E8C0E0BD0100EEF6EA40E07D0B4
:1010B800800EEF6EBB0E03D0600EEF6EEA0EEC6E84
:1010C8001200126EEA6A2F0E1124E96EEFCF14F0A7
:1010D800105005E0176ED8901432172EFCD7030E67
:1010E80014160F14146214D026900FB426802F0EF5
:1010F8001124246E1250DCEC10F026900FB62680D6
:101108002F0E1124246ED8901234DCEC10F013D07A
:1011180026900FB026802F0E1124246E1250DCEC7E
:1011280010F026900FB226802F0E1124246ED8902E
:101138001234DCEC10F011C024F0EA6A2F0E1124EE
:10114800E96EEF50C1EC10F00F380F0B0F6E080E60
:101158001102F3501024136EEA6A980E1124E96EF6
:10116800121CEF160E50020A03E0010A19E02FD0F4
:10117800D89013341B6E0F500BDF01EE00F0D8909F
:101188001334E926EECF15F0EECF16F015501610F1
:101198001EE0EA6A980E1124E96E1250EF1217D079
:1011A800D89013341A6E0F5041DF01EE00F0D8903A
:1011B8001334E926EECF15F0EECF16F015501610C1
:1011C80006E0EA6A980E1124E96E1250EF1201EE59
:1011D80000F0D8901334E92615C0EEFF16C0EEFFD4
:1011E8001200156E105202E0102C0BD012BC09D060
:1011F800EA6A980E1424E96E1550EF1402E0D890AC
:101208001200EA6A370E1424E96E1550EF14D8B4A8
:101218008FD0080E1402F3501324166E105203E0F8
:10122800020E106206D0D89016341B6E1150B0DE34
:101238000AD0104C03D0030E106205D0D890163493
:101248001A6E1150F3DE01EE00F0D8901634E9263C
:10125800EECF18F0EECF19F01050020A07E0010A9D
:1012680010E0030A37E0010A40E060D01850191076
:1012780008E1EA6A2F0E1424E96E1550EF12D8908F
:101288001200EA6A980E1424E96E1550EF144EE124
:10129800EA6AA80E1424E96E1550EF1405E0090E49
:1012A800185E000E195A06D0EA6A2F0E1424E96E49
:1012B8001550EF1A01EE00F0D8901634E92618C040
:1012C800EEFF19C0EEFFEA6A980E1424E96E155075
:1012D800EF122CD01850191008E1EA6A2F0E1424C6
:1012E800E96E1550EF12D8901200EA6AA80E14247D
:1012F800E96E1550EF1405E0090E185E000E195A34
:1013080006D0EA6A2F0E1424E96E1550EF1201EE8A
:1013180000F0D8901634E92618C0EEFF19C0EEFF89
:10132800EA6A980E1424E96E1550EF12D88012005C
:101338001050020A07E0010A05E0030A09E0010A61
:1013480007E013D0EA6A980E1424E96E151CEF160C
:10135800EA6A980E1424E96E1550EF1406E1EA6A59
:101368002F0E1424E96E151CEF16D8901200166E75
:101378000F0E1314176E1338070B186E020A02E0CB
:10138800186629D0080E1502F3501424196E175246
:1013980006E0D89019341B6E1750FADD16D0020EED
:1013A800186209D001EE00F0D8901934E926090E28
:1013B800EE6EEF6A0AD0186608D001EE00F0D890F9
:1013C8001934E926010EEE6EEF6AEA6A980E1524C2
:1013D800E96E1650EF1212000B500924E96E0C50FA
:1013E8000A20EA6EEFCF12F012AC2DD012AA28D044
:1013F8000D06000E0E5A0D500E1021E00BC013F012
:101408000CC014F0132A000E142213500F6205D0DA
:101418001450106202D0136A146A13500924E96E3A
:1014280014500A20EA6EEFCF11F0030E116402D0B7
:10143800110E1160FF0C0D2A000E0E220BD0000CAD
:10144800060E116E07D012AA03D0040E116E02D038
:10145800020E116E126A0B500924E96E0C500A2014
:10146800EA6EEF50121A0B2A000E0C220B500F6274
:1014780005D00C50106202D00B6A0C6A1104136E6E
:10148800135226E00D06000E0E5A0EBE03D00D5064
:101498000E10D8B4000C0B500924E96E0C500A2029
:1014A800EA6EEFBEFF0C0B500924E96E0C500A20BF
:1014B800EA6EEF50121A0B2A000E0C220B500F6224
:1014C80005D00C50106202D00B6A0C6A1306D8D7EC
:1014D800123C02D011501200FF0C166E1338030B89
:1014E800176E19B249D0199415BC19841F0E151618
:1014F800175005E0010A10E0030A30E03CD019A4B7
:1015080005D016501426000E152269D0D890163032
:101518001426000E152263D019B405D016501426CF
:10152800000E152205D0D89016301426000E15226C
:1015380019B009D0159A159815B61588158615A8E5
:101548004ED015964CD01588158A19A448D0010E8E
:10155800161616501588D8B4159841D0158AD89003
:1015680016301426000E1522010E16161650158870
:10157800D8B4159834D012003F0E1516175005E050
:10158800010A0EE0030A1DE029D0159615B8158644
:10159800159815BA1588100E13BC151A159A1FD070
:1015A800100E13BC151A159615B8158619B006D065
:1015B800159A158615A813D0159611D01588158A71
:1015C8000ED0D88015AED890153214321598D8B0F0
:1015D8001588158A080E13BC151A01D01200D89068
:1015E80014361536D8901432186A6950E96E020E0E
:1015F8006A24EA6EB00E1710EF6E1850D0DB186E22
:101608006950E96E020E6A24EA6E14C0EFFF1850A2
:10161800C6DB186E6950E96E020E6A24EA6E15C0C0
:10162800EFFF1850BCDB186E6950E96E020E6A2491
:10163800EA6E181CEF6E000EB2DB140E9FD4085031
:101648000914FF0AD8B4120010EEB0F00D6A080EA3
:101658000D6038D0E6CF0AF0E6CF0BF00BAE30D0F5
:101668000BAC2ED0070E0B1624EE00F0200E0D0248
:10167800F350D926106A010E0E6E0E5221E0DFCF0C
:101688000CF00C38030B13E108500A6210D0095013
:101698000B620DD001EE80F06550E9262690EFBA76
:1016A80026803F0E0D24246E0E50DCEC10F0040E44
:1016B800D926102A0A2A000E0B22D8900E36DDD71A
:1016C8000D2AC5D712001C6ED9CF21F0DACF22F02F
:1016D80024EE00F0200E1B02F350D926040E1A0245
:1016E800F350D926DECF1EF023B01DD01E38030BD1
:1016F8001962E2D0195005E123A2DED0239223B467
:101708002382269023B22680370E1B24246E1C5079
:10171800DCEC10F0EA6A470E1B24E96E1C50EF124D
:10172800140E2CDCC9D01966C7D023A2C5D01AB0B4
:1017380007D0EA6A980E1B24E96E1C1CEF1608D025
:10174800EA6A980E1B24E96ED8901C30FF0AEF163F
:101758001AB027D0268023B42690370E1B24246E77
:101768001C50DCEC10F0268023B426902F0E1B248E
:10177800246E1C50DCEC10F0269023B42680370E23
:101788001B24246ED8901C34DCEC10F0269023B473
:1017980026802F0E1B24246ED8901C34DCEC10F00D
:1017A8007FD023B41FD02690370E1B24246E1C50E4
:1017B800DCEC10F026902F0E1B24246E1C50DCEC61
:1017C80010F02690370E1B24246ED8901C30DCECC9
:1017D80010F026902F0E1B24246ED8901C30DCECC1
:1017E80010F05ED0DFCF1FF01F5006E0050A04E0BE
:1017F8000F0A02E0050A27E126901FB22680370E5D
:101808001B24246E1C50DCEC10F026901FB226809E
:101818002F0E1B24246E1C50DCEC10F026901FB0F9
:101828002680370E1B24246ED8901C30DCEC10F078
:1018380026901FB026802F0E1B24246ED8901C30B3
:10184800DCEC10F02DD02680370E1B24246E1C50A3
:10185800DCEC10F02680370E1B24246ED8901C3048
:10186800DCEC10F0040ED95E5F0EDF1417E0060EF4
:101878001A14206E080E1B02F35020241D6E01EE70
:1018880000F0D8901D34E926010EEE6EEF6AEA6A80
:10189800980E1B24E96ED8901C30EF12040ED9263E
:1018A8001BC024F0EA6A2F0E1B24E96EEF50C1EC2E
:1018B80010F0140EC2EC07F021C0D9FF22C0DAFFE5
:1018C8001200086E50DA01EE80F06550E926D890D3
:1018D800EF340F6E48DA01EE80F06550E9260F0EFE
:1018E800EF14106ED89010320F3201EE80F0655070
:1018F800E9261590EFBC15800850020A05E0030A96
:1019080008E0010A19E02DD015B02ED00F68106834
:10191800FF0C15B029D0EFBA02D0EFA804D0EFAA77
:1019280005D0EFA803D00F681068FF0CEFAA02D00B
:10193800EFA8EF88EF8C18D015A003D00F681068B7
:10194800FF0CF80E0F5C030E10580EE3FC0E0F5C34
:10195800030E105809E20FC016F010C017F0D6D9C0
:1019680003D00F681068FF0C10EEB0F0096A080E7B
:101978000960C3D1E6CF11F0E6CF12F012BEBBD199
:1019880024EE00F0200E0902F350D926DD501596FA
:1019980012BA1586159A12BC158A070E12160E6A07
:1019A8000850010A06E0010A04E0020AD8B4EDD0A2
:1019B800A2D1010E0D6E0D52D8B49DD1DCCF0BF023
:1019C8000F50116258D01050126255D001EE80F0BD
:1019D8006550E9261592EFB8158201EE80F0E926E8
:1019E8001594EFBA1584086607D0040EDFBE151AE1
:1019F800159C15B4158C06D0020EDFBE151A159C61
:101A080015B2158C030E0B14010A07E0030A08E04F
:101A1800010A08E0030A2FE005D015BC03D02BD03B
:101A280015BC29D015B616D015AA14D00EA012D000
:101A380008C019F0239015B62380239215B223828B
:101A4800238415B423940EC01AF009C01BF00D505E
:101A58003ADE11D008C019F0239015B623802392DE
:101A680015B22382239415B423840EC01AF009C03A
:101A78001BF00D5028DE030ED926DFAE77D0300ECE
:101A8800DF140C6E0C38086271D0070EDD14146E6A
:101A9800DECF13F00F50136269D01050146266D075
:101AA80001EE80F06550E9261592EFB8158201EE37
:101AB80080F0E9261594EFBA1584086607D0040E5D
:101AC800DFBC151A159C15B4158C06D0020EDFBCA8
:101AD800151A159C15B2158CD8900B32D8900B326C
:101AE800030E0B14010A05E0030A06E0010A06E0EA
:101AF8003DD015BC03D03AD015BC38D0D8900B32A5
:101B0800D8900B32030E0B160B5007E0010A02E0C7
:101B1800030A2CE1159215B4158215B616D015AA2C
:101B280014D00EA012D008C019F0239015B6238047
:101B3800239215B22382238415B423940EC01AF07D
:101B480009C01BF00D50BFDD11D008C019F023905B
:101B580015B62380239215B22382239415B42384C7
:101B68000EC01AF009C01BF00D50ADDD0E2A112A67
:101B7800000E122215AA06D015B604D00EA002D067
:101B88001106125AD8900D3616D7010E0D6E0D5249
:101B9800D8B4B1D00F5011623FD0105012623CD06F
:101BA800DCCF0BF001EE80F06550E9261592EFB816
:101BB8001582020EDFBE151ADD50030E0B14010A42
:101BC80007E0030A08E0010A08E0030A25E005D057
:101BD80015B203D021D015B21FD001EE80F06550A8
:101BE800E926EFAA03D00E2AD8900D3608C019F0BE
:101BF8002390239215B2238223940EC01AF009C0B1
:101C08001BF00D5060DD01EE80F06550E926EFAA6B
:101C180003D00E06D8900D321598DCCF0BF0030ECA
:101C2800D926000EDA22DFAE5CD0300EDF140C6E3F
:101C38000C38086256D00F0EDD14146EDECF13F088
:101C4800D890143213320F5013624BD010501462D4
:101C580048D0DD5001EE80F06550E926EFBA03D098
:101C6800DEA003D03ED0DEA03CD001EE80F065506F
:101C7800E9261592EFB81582020EDFBC151AD89026
:101C88000B32D8900B32030E0B14010A05E0030A3D
:101C980006E0010A06E025D015B203D022D015B21D
:101CA80020D0D8900B32D8900B32030E0B160B5065
:101CB80005E0010A07E0030A05E013D0159415B200
:101CC800158415820BC019F02390239215B2238234
:101CD800239415B423840EC01AF009C01BF00D50CC
:101CE800F2DC0E2AD8900D36157815B896D7112A39
:101CF800000E12224CD7092A3AD60F50120033D8B8
:101D0800C2A503D079840A0E766E1200C2A72AD023
:101D180001EE80F06550E926EFB824D0030E1614C2
:101D2800196ED890193601EE80F06550E926EFBAA1
:101D38001980080E196016D0E26AD8901934B10FCC
:101D4800E16EE7AE07D0EA6A470E1924E96EEF683C
:101D5800798208D0C2A906D0EA6A470E1924E96E2A
:101D6800EF687982120001EE80F06550E926EF6A8B
:101D7800652A600E656201D0656A12006750E96ED7
:101D8800020E6824EA6EEF6A672A000E6822676608
:101D980005D0020E686202D0676A686A12001A6E7D
:101DA8006950E96E020E6A24EA6EEF501A1A692A1F
:101DB800000E6A22696605D0020E6A6202D0696A5C
:101DC8006A6A1A501200B00E126E136A146AB50EBF
:101DD800156E45DA116A106A040E10600ED0136E83
:101DE8001150126E400E1124146EB50E156A15228C
:101DF80036DA400E1126102AEFD7CADA268EFBDA19
:101E0800269E1200B0DFC2A31200ADDF01EE80F003
:101E18006550E9267C0EEF626FD0A5DF01EE80F0F9
:101E28006550E926EFCF0CF09EDF9DDF01EE80F0D4
:101E38006550E926EFCF09F096DF01EE80F0655096
:101E4800E926D890EF34086ED88009AED8900932C8
:101E580008323F0EC0150B6EC1C00AF079B606D025
:101E680008500A6249D009500B6246D07CDF7BDFFC
:101E7800FC0E0C14200A0BE0080A09E0040A15E01D
:101E88004C0A21E0080A1FE00C0A2AE035D079A69E
:101E980009D0C2AF07D00CC00DF008C00EF009C0C1
:101EA8000FF02BD8010E89D827D079B607D00CC0EF
:101EB8000DF008C00EF009C00FF01FD8C2AF1CD03B
:101EC8007F0E7BD819D079A606D0D1D8C2AF14D04E
:101ED800400E73D811D0C2AF0FD0000E6ED80CD000
:101EE80079B606D0C4D8C2AF07D0400E66D804D0A1
:101EF800C2AF02D0000E61D8120015EE00F0E70E56
:101F0800E66E0E0EE66E7C0EE66E0DC0E6FF100E57
:101F1800E66ED8900E360F36D8900E320FC0E6FF18
:101F28000EC0E6FFE66A166A01EE80F06550E92603
:101F3800EFCF14F014C018F018380F0B186E13DF19
:101F480001EE80F06550E926EFCF15F015C017F0C7
:101F5800179E14B0178E18500FE1160E17600CD08C
:101F6800B00E1724E96E000E1820EA6EEFCF16F0B7
:101F7800140EC2EC07F013D0160E175C010E185899
:101F88000EE2160E175E000E185A1750E96E040E70
:101F98001824EA6EEFCF16F0140EC2EC07F0149274
:101FA80016BE148214C0E6FF15C0E6FF7F0E161495
:101FB800E66EE66AE66A798C12000D6E0E6A695062
:101FC800E96E020E6A24EA6EB40EEF6E0E50E7DE7A
:101FD8000E6E6950E96E020E6A24EA6E6F0EEF6E9D
:101FE8000E50DDDE0E6E6950E96E020E6A24EA6E4E
:101FF8000DC0EFFF0E50D3DE0E6E6950E96E020E73
:102008006A24EA6E0E1CEF6E000EC9D6096AABDEB2
:1020180001EE80F06550E9266F0EEF6227D079ACAB
:1020280025D0799C15EE00F06950E96E020E6A24FD
:10203800EA6EE6CFEFFF0950B2DE096E020EE75CEA
:10204800086E6950E96E020E6A24EA6EE6CFEFFF69
:102058000950A5DE096E082EF4D76950E96E020E04
:102068006A24EA6E091CEF6E000E99D6120001EE82
:1020780080F06550E926EFCF0FF075DE01EE80F0B5
:102088006550E926EFCF0EF00E9E0FB00E8E6BDE78
:1020980001EE80F06550E926EFCF0DF00D9E0FB2EE
:1020A8000D8E0F380F0B0F6E140E0E6202D00F52EA
:1020B80005E0150E0E620BD00F6609D0AA0E0D6250
:1020C80001D081DEA10E5E6E140EC2EF07F00F5034
:1020D80013E1140E0E6010D0B00E0E24E96E000E3F
:1020E8000F20EA6E0DC0EFFF04000EC019F00FC0FC
:1020F8001AF00D5078D81BD0160E0E5C010E0F5832
:1021080015E2160E0E5E000E0F5A0E50E96E040E02
:102118000F24EA6E0DC0EFFF0400400E0E24196E66
:10212800000E0F201A6E0D505ED801D0120030D963
:102138000F500AE1100E0E6007D0010E0E14010AAE
:1021480003E1268E58D9269E510E5E6E140EC2EFFC
:1021580007F0196EF00E801619508026899881CFE5
:102168001AF01A9082BA1A808988EA6A900E19249D
:10217800E96EEF501A1A1A501200256EEA6A900E8C
:102188002424E96EEF50251A010E9316949A25C05F
:1021980081FF25A0829A25B0828AF00E8016080E4B
:1021A8002424802689988988FE0E9312948A120026
:1021B800256E24C0E9FFEA6AD890EF14D8A4D88025
:1021C80026A003D02550EF1202D0251CEF161200CE
:1021D800A6B2FED71CC0A9FF1DC0AAFFA69EA69C3A
:1021E800A680A85012001B6E19C01CF01AC01DF062
:1021F800EFDF1B1832E0A6B2FED71BC0A8FF19C03C
:10220800A9FF1AC0AAFFA69EA69CA684F29E550EF8
:10221800A76EAA0EA76EA682F28EA694632A000E57
:102228006422E90E635C030E64580EE3636A646A11
:10223800612A000E6222F10E615C030E625804E30B
:10224800400E616E010E626E19C01CF01AC01DF0BE
:10225800BFDF1B1802E0D8901200D8801200A68EAB
:10226800A69CF86A1550F76EC00E1414F66E12C0CC
:10227800E9FF13C0EAFF400E166E0900F552F5CFCC
:10228800EEFF162EFAD712000AC0F6FF0BC0F7FFB2
:10229800F86AA68EA69C0800F55012000F0EC16EB3
:1022A800070EB46E300E806EC00E926E816A93680F
:1022B800D50E826EEA0E946ED0A60AD0D0A408D0AD
:1022C80000EE00F00F0EEE6AEA62FDD7E9AEFBD72A
:1022D800F19CF298F2924A0EAF6EAC84AC98AB8E39
:1022E8009D989D9AAC9AAB98D56ACD6A9E909D8030
:1022F800480ECA6ECC6A7C0ECB6E9E929D82B16AE5
:102308001200140E0A6EB50E0B6EBEDF096E140EA7
:102318001C6E1D6A5DDF091809E009C0A8FFA684C4
:10232800550EA76EAA0EA76EA682A69400EEB0F070
:10233800076A086AA68407C01CF008C01DF048DFB9
:10234800EE6E550EA76EAA0EA76EA682072A000E7D
:102358000822085003E1150E0764EDD704EE00F0DB
:10236800400E076E086A07C01CF008C01DF030DF79
:10237800EE6E550EA76EAA0EA76EA682072A000E4D
:102388000822400E075C010E0858EDE3A6941200DF
:102398006068010E126E10EEB0F0136A080E13603A
:1023A80029D0EA6A900E1324E96EEF6A010E156EC1
:1023B80024EE00F0200E1302F350D926E650E6BEB4
:1023C80003D0D92A121C6016176A200E17600ED087
:1023D800DFAE06D0EA6A900E1324E96E1550EF12AC
:1023E800D8901536040ED9261726EFD7D89012366E
:1023F800132AD4D71200010E9316949A60C081FF55
:1024080060A0829A60B0828A899A898AFE0E9312A5
:10241800948A8B981C6E030E1D6EDADE616E1C6842
:10242800030E1D6ED5DE626E1890F10E615C030E10
:10243800625805E31880400E616E010E626E269C9C
:10244800C2B1268C26AC15D026AE05D061C016F0D8
:1024580062C017F005D06128166E000E6220176E54
:10246800F10E165C030E175804E3400E166E010EAB
:10247800176E070E126E12BE74D0E26AD89012342C
:10248800B10FE16E26AC60D018B002D026AE02D0F3
:10249800136A0AD0125061241C6E000E12BEFF0E81
:1024A80062201D6E95DE136E040012501624196EFC
:1024B800000E12BEFF0E17201A6E135094DEE7BEF0
:1024C8003DD0EA6A370E1224E96E13C0EFFFE7AA7F
:1024D8002FD0EA6A2F0E1224E96E13C0EFFF12C044
:1024E80024F0EA6A2F0E1224E96EEF5046DE020E3F
:1024F800156E010E146E080E146026D0030E131408
:10250800030A0BE1196A23802382238414C01AF07A
:1025180012C01BF0155067EC0BF0D8901332D8900E
:102528001332D8901536D8901536020E1426E3D7F4
:10253800EA6A470E1224E96EEF6806D0EA6A3F0E8F
:102548001224E96E13C0EFFFE7AE09D0125001DE86
:10255800136EEA6A370E1224E96E13C0EFFF1206F3
:102568008AD716C061F017C062F00400FE0E196E1B
:10257800030E1A6E615037DE04001968030E1A6ED6
:04258800625031D696
:10B50000008008801080188020802880308038805B
:06B51000E7100F000657D2
:10B54000230000002300000023000000230000006F
:10B55000230000002300000023000000230000005F
:10B56000230000002300000023000000230000004F
:10B57000230000002300000023000000230000003F
:10B58000230000002300000023000000230000002F
:10B59000230000002300000023000000230000001F
:10B5A000230000002300000023000000230000000F
:10B5B00023000000230000002300000023000000FF
:10B5C00023000000230000002300000023000000EF
:10B5D00023000000230000002300000023000000DF
:10B5E00023000000230000002300000023000000CF
:10B5F00023000000230000002300000023000000BF
:10B6000023000000230000002300000023000000AE
:10B61000230000002300000023000000230000009E
:10B62000230000002300000023000000230000008E
:10B63000230000002300000023000000230000007E
:0200000400F00A
:100000000080088010801880208028803080388010
:06001000E7100F00065787
:100040002300000023000000230000002300000024
:100050002300000023000000230000002300000014
:100060002300010023000200230000002300000001
:1000700023000000230000002300000023000000F4
:1000800023000000230000002300000023000000E4
:1000900023000000230000002300000023000000D4
:1000A00023000000230000002300000023000000C4
:1000B00023000000230000002300000023000000B4
:1000C00023000000230000002300000023000000A4
:1000D0002300000023000000230000002300000094
:1000E0002300000023000000230000002300000084
:1000F0002300000023000000230000002300000074
:100100002300000023000000230000002300000063
:100110002300000023000000230000002300000053
:100120002300000023000000230000002300000043
:100130002300000023000000230000002300000033
:020000040020DA
:080000000507000100010001E9
:020000040030CA
:08000000FF021F08FF8181FFD0
:00000001FF
